:1000000000308A00822800000A108A100A11820734
:1000100025344C34753420346D3473340A340D3443
:10002000003423308400831300080319282801308A
:10003000F800BF30F7006400F70B1B28F80B1928F5
:100040004A30F700F70B222800006400800B1728C5
:100050000034AB010408AA002B10831B2B14240EC0
:10006000F038A600A607E23EA700323EA900240809
:100070000F39A707A707A907E93EA800A807A807FF
:10008000230E0F39A807A907A80DA90DA909A90DC5
:1000900023080F39A907A60D0730A5000A30A907C4
:1000A000A803031C4F28A807A703031C5328A7076E
:1000B000A603031C5728A607A503031C5B282530AD
:1000C0008400831307302A052A1384072930040289
:1000D00003192A170008F700031D76282A1B762823
:1000E0002A1A7E28AA19762820307928AA152A12D9
:1000F0003030F70777080C1E7B289900840A2A1FE6
:100100006628F628840183131F308305193083166F
:100110009900A630980090308312980083161F141F
:100120009F141F159F1107309C00FF308312A00001
:1001300083161F149F141F159F1183121F108316FF
:10014000091283129412A0122008831687008312CA
:1001500020162008831687008312A011200883161A
:100160008700013083129400003083169400010848
:10017000C73908388100831290010030F8009200DE
:1001800000308316920006309C0005080338850075
:1001900064000230F700F70BCB28CE281C0883122E
:1001A0000D13803083169D008312A201A1018316D6
:1001B0001C1FE3288312A10A0319A20A0130A3001D
:1001C0001120D72883161C1BEE288312A10A0319BD
:1001D000A20A0130A30011208316E3281030840006
:1001E00083122208A4002108A30029280330A300B9
:1001F00023080420A30AF70077080C1EFD289900A5
:0C02000008302302031DF828D5286300F5
:02400E00393F38
:00000001FF
